:100000000C9443020C9460020C9460020C94600205
:100010000C9460020C9460020C9460020C946002D8
:100020000C9460020C9460020C9429210C94FD2124
:100030000C945C1B0C9460020C9460020C946002A3
:100040000C9460020C9460020C9460020C946002A8
:100050000C9460020C94E31B0C9460020C946002FC
:100060000C9460020C9460020C9460020C94600288
:100070000C9460020C9460020C9460020C94600278
:100080000C9460020C9460020C9460020C94600268
:100090000C9460020C9460020C9460020C94600258
:1000A0000C9460020C9460020C946002290014000D
:1000B0001A000800150017001C0018000C001200A0
:1000C00013002A002B0004001600070009000A0094
:1000D0000B000D000E000F0033003400E1001D0086
:1000E0001B00060019000500110010003600370043
:1000F000380028000351E000E300E20001512C0029
:100100002C0002515000510052004F0035021E02D7
:100110001F022002210222022302240225022602BB
:1001200027022A004C003A003B003C003D003E0004
:100130003F002D022E022F0230023102010040004A
:1001400041004200430044004500010001004A0014
:100150004D0001000100010001000100010001004B
:1001600001000100AB00AA00A900AE0035001E008E
:100170001F0020002100220023002400250026006B
:1001800027002A004C003A003B003C003D003E00A6
:100190003F002D002E002F003000310001004000F4
:1001A00041004200430044004500010001004B00B3
:1001B0004E000100010001000100010001000100EA
:1001C00001000100AB00AA00A900AE000100005C24
:1001D000015C0100010001000100010001000100BB
:1001E00001004C00010001000100010001000100BC
:1001F00001000100010001000100010001000100F7
:1002000001000100010001000100010001000100E6
:1002100001000100010001000100010001000100D6
:1002200001000100010001000100010000000000C8
:10023000000000002A2B2800000000000000000041
:100240000000000000000029000000002C1E3420E7
:10025000212224342627252E362D3738271E1F200D
:100260002122232425263333362E37381F04050652
:100270000708090A0B0C0D0E0F1011121314151696
:100280001718191A1B1C1D2F3130232D3504050694
:100290000708090A0B0C0D0E0F1011121314151676
:1002A0001718191A1B1C1D2F3130354C0000000087
:1002B000000000000000000000000000000000003E
:1002C000000000000000000000000000000000002E
:1002D0007E0F00D4FFFFFFC7000000780E0343002D
:1002E0006F006E0074007200610000000E03430096
:1002F00061007200740065006C00000004030904D2
:1003000009025B00030100A0FA09040000010301D7
:1003100001000921110100012240000705810308A5
:10032000000109040100020300000009211101007D
:100330000122220007058203200001070503032094
:10034000000109040200010300000009211101005D
:100350000122B600070584032000011201000200FB
:10036000000008544301000100010200010660FF83
:100370000961A1010962150026FF00952075088119
:10038000020963150026FF00952075089102C0053B
:10039000010902A10185020901A10005091901292C
:1003A000081500250195087501810205010930092C
:1003B000311581257F95027508810609381581253B
:1003C0007F950175088106050C0A38021581257F85
:1003D000950175088106C0C005010980A10185034A
:1003E00019012AB700150126B70095017510810083
:1003F000C0050C0901A101850419012AA0021501FB
:1004000026A002950175108100C005010906A10111
:100410008506050719E029E71500250195087501EE
:1004200081020507190029EF1500250195F07501D6
:1004300081020508190129059505750191029501AB
:1004400075039101C005010906A101050719E029FD
:10045000E715002501950875018102950175088150
:10046000010507190029FF150026FF0095067508EC
:10047000810005081901290595057501910295016D
:1004800075039101C00011241FBECFEFDAE0DEBF7B
:10049000CDBF11E0A0E0B1E0E6E2F9E402C00590D2
:1004A0000D92A839B107D9F722E0A8E9B1E001C05F
:1004B0001D92A73AB207E1F70E945B110C946824E1
:1004C0000C94000084E0089581E0089581E008958F
:1004D0000E946602089508950E946B020895A5E0A7
:1004E000B0E0E5E7F2E00C94D42349835A833091DD
:1004F0009F0189819A81311119C0662399F02223C5
:1005000089F00E945E08182F682F89819A810E94C5
:100510003A0869817A81812F0E9447182596E3E085
:100520000C94F0230E944C08182FF3CF0E945E0811
:1005300069817A81F1CFFC01262F4081518162814E
:10054000738184810E946F02089581E00895CF93A2
:10055000DF93EC0160E00E949B02BE010E946C02EE
:10056000DF91CF910895E1E0F0E0DF0102C0AA0F32
:10057000BB1F6A95E2F7BD01DF0102C0AA0FBB1FD6
:100580004A95E2F76A2B01C0EE0F2A95EAF7962FFB
:100590009823961302C08E2B0895E0958E2308951C
:1005A000242F462F682F8091B2010E94B3020E942F
:1005B0009A0708950E94001008950E94041008955B
:1005C00008950E942C070E94E0022FEF84E39CE034
:1005D000215080409040E1F700C0000008950E9443
:1005E000E1020E94071C08950E94E1020E94181C6B
:1005F00008950F931F93CF93DF938C0161E00E94C6
:100600009B02EC01B8010E945114811106C080E0E8
:10061000DF91CF911F910F910895B801CE010E94F3
:1006200068028823A1F3B801CE010E948D198823A6
:1006300071F3B801CE010E944015882341F3B8013F
:10064000CE010E94FF18882311F3F80182818823CC
:1006500061F0CA35FDE5DF0701F158F4C115ECE59D
:10066000DE0791F0CE3DDC4591F0C8010E946402A6
:10067000CFCFCC358DE5D80769F090F0C73ADD458E
:10068000A1F70E94F402C3CF0E94EF02C0CF0E94E4
:10069000170DF7CF0E94510CE8CF0E945B0CE5CFFD
:1006A0000E945F0CE2CF0E94381B0E9470030895E5
:1006B0000E9474030E943D1B089508950E945D03EB
:1006C000089581E008950E94610308950895CF93ED
:1006D000C82F0E945E038C2F0E946303CF91089560
:1006E00080E00E94670308950E94E9190E94670351
:1006F0000895CF930E94E919C82F80919A018C1711
:1007000079F0C0939A010E94C81B60939B0170937B
:100710009C0180939D0190939E018C2F0E94670302
:10072000CF910895ABE0B0E0E8E9F3E00C94D52375
:100730004F83588769877A878B8761110E949C0B4A
:100740001E821D8285E0FE013796DE011196019022
:100750000D928A95E1F78C819D81892B61F4498105
:100760005A816B817C818D819E810E94C50A2B9666
:10077000E2E00C94F12389819A8189238F3F79F3F8
:10078000CE0101960E94A5028111E9CFF0CFFC01B4
:10079000808191810E948B080895CF93C82F882370
:1007A000C9F08238C9F40E94E91981FD13C089E3B8
:1007B0000E94540B0E94BD0B2FEF87EE93E0215057
:1007C00080409040E1F700C0000089E30E945C0B8C
:1007D0000E94BD0BCF9108958338A1F40E94E919BE
:1007E00080FDF8CF83E50E94540B0E94BD0B2FEFD4
:1007F00081EE94E0215080409040E1F700C000007D
:1008000083E5E4CF8438A1F40E94E91982FDE2CFA8
:1008100087E40E94540B0E94BD0B2FEF81EE94E001
:10082000215080409040E1F700C0000087E4CECF27
:100830008CEF8C0F813A90F46C2F80910001909195
:1008400001010E945E1A882329F08C2F0E945C0B04
:100850000E94BD0B8C2F0E94540BBACF80E28C0FEC
:10086000883048F4C77081E001C0880FCA95EAF764
:100870000E947F0BADCFEBE5EC0FE33040F4F0E0EE
:10088000EB5BFE4F808190E00E941E1AA3CFE8E54B
:10089000EC0FE73150F4F0E0EE0FFF1FE95EFE4F82
:1008A000808191810E94341A95CFC03F08F492CF85
:1008B0008C2F0E94DF110E94B2128CCF882309F482
:1008C00055C0823879F40E94E91981FF4FC089E34D
:1008D0000E94540B0E94BD0B89E30E945C0B0E9496
:1008E000BD0B0895833859F40E94E91980FF3EC07A
:1008F00083E50E94540B0E94BD0B83E5EECF843844
:1009000059F40E94E91982FF31C087E40E94540B18
:100910000E94BD0B87E4E1CF9CEF980F913AE8F27B
:1009200090E2980F983050F4877091E001C0990FD1
:100930008A95EAF7892F0E94850BD1CF9BE5980F06
:10094000933028F490E080E00E941E1A089598E504
:10095000980F973128F490E080E00E94341A0895AF
:10096000803F20F00E9439120E94B21208951F9316
:10097000CF93DF93182FEB010E94CD03209739F41A
:10098000812F0E945E04DF91CF911F9108958FE91E
:100990009FE00197F1F700C000002197EFCF70E0D2
:1009A00060E0893311F460E570E00E94B7040895B7
:1009B000882321F00E947F0B0E94BD0B089588239D
:1009C00021F00E94850B0E94BD0B0895B0E0A0E0CD
:1009D000ECEEF4E00C94CE236C01D62FC72FFC0173
:1009E0001281F580F2949FE0F9220E94750BE82EA7
:1009F0008823B9F0E12E1123A1F08C2F807F803461
:100A000021F080E28D0F8830D0F08091850282FF46
:100A100016C082E00E94200C0E94750B91E0E82E27
:100A2000E926BC2EB2948FE0B822FBE0FB1508F457
:100A300068C0EB2DF0E0E659FB4D0C94B823E12C97
:100A4000F0CF0C2F0F70C07F11F00295007F1123A3
:100A500099F0002359F080E28D0F883010F0D11109
:100A600007C0802F0E947F0B0E94BD0B8D2F41C0BD
:100A7000802F0E948F0BF8CF8D2F0E945E040023E1
:100A800009F43FC080E28D0F883010F0D11104C00E
:100A9000802F0E94850B03C0802F0E94950B0E941F
:100AA000BD0B2FC00C2F0F70C07FC03211F002950C
:100AB000007FDD2381F0D13009F463C0112309F4F4
:100AC0006DC0FF2009F463C0F601858180FFCECFA1
:100AD0008F7085835CC08091850282FD33C01123B5
:100AE00059F0002329F0802F0E947F0B0E94BD0B3C
:100AF00080E00E94CD0305C080E00E945E040111E9
:100B0000C7CFEB2DE850FF0B349720F40E94E91972
:100B10000E946703EE2089F00E94710B80FD0DC0DA
:100B2000F60112820E946B0B0E94AE07C6010E9462
:100B3000EC060E946B0B0E94BA07CDB7DEB7E9E066
:100B40000C94EA23112389F0F11006C00E949F0B38
:100B5000802B0E94D804D5CF21E0F212F7CF0E945B
:100B60009F0B802B0E94A60BCCCFF11006C00E94D9
:100B7000B30B802F0E94DF04C4CF31E0F31609F2DB
:100B8000F6CF112331F085E08F1508F4BACF802F0E
:100B9000E0CF94E09F1508F4B4CFEBCFFF2049F3EA
:100BA000D93349F4FFEF27EE33E0F15020403040D5
:100BB000E1F700C000008D2F0E945E04A2CF8C2FB1
:100BC00086958695837069F0813009F09ACF8D2FD4
:100BD0009C2F9370111102C090E080E00E94341AA3
:100BE00090CF8D2F9C2F9370111102C090E080E068
:100BF0000E941E1A86CF8D2F112329F00E94DF112B
:100C00000E94B2127ECF0E943912FACF8C2F8370CD
:100C100079F5111176CF4D2F429546954770440FC7
:100C2000440F8D2F8F70042E01C0880F0A94EAF7AD
:100C30002D2F2071D4FF07C02FE030E001C0220F1C
:100C40004A95EAF72095C695C695C370822BC230A7
:100C500049F058F4C13019F00E94880752CF0E9421
:100C600082074FCF0E948E074CCF0E947F0749CF4B
:100C70008695112311F08C2F8170882309F441CFC0
:100C80004D2F429546954770440F440F8D2F8F701E
:100C9000042E01C0880F0A94EAF72D2F2071D4FF8B
:100CA00007C02FE030E001C0220F4A95EAF72095F7
:100CB000C695C695C370822BC23049F058F4C13036
:100CC00019F00E94D9071DCF0E94D3071ACF0E94A6
:100CD000DF0717CF0E949A0714CFCF70112329F096
:100CE0008C2F0E94AE078D2F34CF8D2F0E94DF04F2
:100CF0008C2F0E94BA0705CFD23F51F160F4D03F4C
:100D0000B9F0D13F81F0112309F449C0F110AECE02
:100D10008C2F8F7121C0D33F11F1D43FA1F7809167
:100D2000850282FD26C08C2F8F71112311F314C010
:100D3000112349F084E08F1508F4E3CE8C2F8F71D6
:100D40000E94C707DECE95E09F1508F4DACEF6CFF5
:100D50008C2F8F711111CDCF0E94AE07D2CE1123EF
:100D600029F08C2F8F710E94A507CBCE0E94A1077E
:100D7000C8CE112349F0CF718C2F0E94AE0763E0DB
:100D80008C2F0E94020CBDCE81E00E94200CE1E07D
:100D9000EF1508F0B6CE82E00E94200CB2CEF11022
:100DA000FFCE8C2F8F71A5CF0F931F93CF93DF931F
:100DB000EC01688179818A810E9496088C010E94E9
:100DC000E5070E947E07B801CE010E94E604DF918C
:100DD000CF911F910F910895CF93DF93EC018B81F9
:100DE0009C81892B29F08881998189238F3F51F437
:100DF000DF91CF910895CE010E94D406CE010E94CA
:100E0000A702F6CFCE010E94F9028111F4CF0E9411
:100E1000750B882369F38A81882351F380918502B9
:100E200082FFE6CF82E00E94200CE2CF90E080E0DB
:100E30000E941E1A90E080E00E94341A0E949C0BCF
:100E40000E94BD0B0E94CE120E94B21208950E9411
:100E5000640B0E94160708950E948C0B0E942707BE
:100E6000089592959F70963091F058F4925F9F701C
:100E7000923058F4803F19F030F4883E30F481E02D
:100E800008959A5FF4CF843FD1F380E00895883EBF
:100E9000B0F3813FD1F7F3CFFC0183819481892B9B
:100EA00029F08081918189238F3F11F480E008959A
:100EB000808191810E948B080E9431070895A5E0EE
:100EC000B0E0E5E6F7E00C94D5232596E2E00C943B
:100ED000F123A6E0B0E0EFE6F7E00C94D5232696E8
:100EE000E2E00C94F12308950E94730708950E9494
:100EF00074078093B3010E941607089508950E9415
:100F0000770708959091B301892B0E947707089580
:100F10009091B30189230E94770708959091B301BE
:100F200089270E94770708950E94730708950E94F9
:100F3000940708950E9497078093B2010E941607B4
:100F4000089580E00E949A07089591E001C0990FEA
:100F50008A95EAF7892F0E949A07089521E030E0E8
:100F600001C0220F8A95EAF78091B201822B0E947C
:100F70009A07089521E030E001C0220F8A95EAF730
:100F800020958091B20182230E949A07089521E062
:100F900030E001C0220F8A95EAF78091B2018227E2
:100FA0000E949A0708959091B201892B0E949A0796
:100FB00008959091B20189230E949A070895909113
:100FC000B20189270E949A0708950895262F277055
:100FD00091E001C0990F2A95EAF723E0769567958D
:100FE0002A95E1F7FB01EE0FFF1FE60FF71FE40F55
:100FF000F51F50E040E0682F70E08191DF0111970C
:101000009B01042E02C0369527950A94E2F72170C1
:1010100021952827292328272C934F5F5F4F4330A2
:10102000510559F70895A82FA77023E09695879545
:101030002A95E1F7FC01EE0FFF1FE80FF91FE60FFD
:10104000F71F50E040E080E0219130E00A2E02C01E
:10105000369527950A94E2F721703327042E01C0B4
:10106000220F0A94EAF7822B4F5F5F4F43305105FE
:1010700059F70895262F943070F48C3060F4682F5F
:1010800070E08CE0989F600D711D112440EA51E0E2
:10109000822F0E94E6070895292F943068F48C303F
:1010A00058F490E060EA71E03CE0239F800D911DD0
:1010B00011240E941308089580E00895CF92DF92D2
:1010C000FF920F931F93CF93DF936C010091B201B6
:1010D0008091B301082BC7E0D0E010E0FC2EC801DE
:1010E0000C2E02C0959587950A94E2F780FD0CC0FE
:1010F0002197A0F7F12C8F2DDF91CF911F910F91A8
:10110000FF90DF90CF900895B6018C2F0E94DE0EE5
:10111000019771F3F0CFCF93DF93EC010E945E084B
:10112000BE010E94DE0EDF91CF9108951F93CF93F1
:10113000DF93EB0190919F01992339F0CB010E943D
:101140008B08DF91CF911F910895882369F0CB011F
:101150000E945E08182F682FCE010E943A08BE0137
:10116000812F0E94DE0EEDCFCB010E944C08182F7C
:10117000F6CF1F93CF93DF93C091B40116E0809117
:10118000B5018C1304C0DF91CF911F910895D0E079
:101190001C9FF0011D9FF00D1124EA54FE4F408169
:1011A000518162817381848195810E9469072196B2
:1011B000C770E5CF4091E6015091E7016091E801E9
:1011C0007091E9018091EA019091EB010E94690719
:1011D00008951F93CF93DF938091EB01807F09F0F7
:1011E00049C08091E801882309F444C08091B4018A
:1011F000C091B5016091E6017091E701A091E9010C
:10120000B091EA01D62FD72316E0C81799F190E0E4
:10121000109711F0DF3F19F401968770F6CF189FF1
:101220009001199F300D1124F901EA54FE4F4181BC
:101230004713F2CF40814613EFCF42814111ECCFEB
:10124000438154814A1B5B0B483C510528F7809130
:10125000EB018F7080618093EB01F901E554FE4F43
:1012600080818F708061808386EE91E00E94EC0621
:101270000E94B908DF91CF911F910895A1E1B0E0DC
:10128000E4E4F9E00C94CD238C0185E0F801DE0163
:101290001D9601900D928A95E1F7F801E28086EEA5
:1012A000C82E81E0D82E6091E9017091EA016115A4
:1012B000710509F44EC19091E6012091E701892F53
:1012C00082238F3F09F445C140815181A380B480BE
:1012D000F090E801F501E61BF70BFF2009F4EAC0E6
:1012E0008091EB01382F307FE83CF10508F0A3C076
:1012F00031116DC0FE2C251316C0941314C0E110DB
:1013000012C08F7080618093EB010E94DA08C601E1
:101310000E94EC068091EB01F80185838F2D619688
:10132000EAE00C94E923A114B10429F0842F852369
:101330008F3F09F027C180E0F82FF170DF2E80FF8A
:101340003CC08091B4012091B50136E0821315C0F4
:101350004D875E878D859E850E948B08292F22955B
:101360002F702230F0F0243018F59F70F1F0F80162
:101370009581907FD1F4D12C1EC090E0389FF00170
:10138000399FF00D1124EA54FE4F6181651306C0A8
:101390006081641303C06281E6120FC001968770FA
:1013A000D5CF9F7011F0882331F3805E883018F319
:1013B000C8010E94EC06FD2CB1CFEE2009F4AECF9F
:1013C0008091EB0181608093EB01F12CA7CF251375
:1013D00006C0941304C0F801EE2009F487C0C801C8
:1013E0000E944C07882319F1EE2009F18091EB014E
:1013F000803270F02091E6013091E70138872F8329
:101400001986BB86AA868C87CE0107960E94EC06B9
:1014100086E0F801A6EEB1E001900D928A95E1F721
:101420000E94E9080E94DA08FF24F39477CFC801EC
:101430000E94EC06F9CF311113C07A2DB98AA88A1F
:101440006E2D89890E945F0786EE91E00E94EC066E
:1014500086E0F60111928A95E9F70E94DA08B5CF85
:1014600025130FC094130DC0E1100BC0F801858344
:10147000C8010E94EC0686E0F60111928A95E9F710
:101480004DCFC8010E944C07882389F2EE2079F2E3
:101490008091EB01803208F4BBCF2091E6013091BE
:1014A000E7013A8329831B82BD82AC828E83CE0101
:1014B0000196ACCFE83CF10508F03EC0FE2CEE20D2
:1014C00009F4B5CF25132AC0941328C08091EB01ED
:1014D00080FD1BC0982F907FC1F0F8018583903F5D
:1014E00031F0982F907F905F8F70892B8583C80192
:1014F0000E94EC0686E0F801A6EEB1E001900D92A4
:101500008A95E1F70E94DA0809CF86E0F801A6EE95
:10151000B1E001900D928A95E1F700CFC8010E94D9
:101520004C07811175CF8091EB0181608093EB01B5
:10153000C8010E94EC06F2CE7A2DB98AA88A6E2DD7
:1015400089890E945F0786E0F60111928A95E9F782
:10155000D9CFEE2009F46BCFC8010E944C07F82EBA
:10156000882309F464CF86E0F801A6EEB1E001908B
:101570000D928A95E1F786EE91E00E94C7030E94E2
:10158000E908C0CF81E08E25D7CEACE0B0E0EBEC2F
:10159000FAE00C94D4234F83588769877A878B8726
:1015A0009C87CE0107960E943E09882369F08A85B0
:1015B0009B85892B39F04F815885842F85238F3F58
:1015C00009F06BC016E05FC086E0FE013796DE01D1
:1015D000119601900D928A95E1F78A859B85892B5A
:1015E00089F388859F8189238F3F61F32091B5011D
:1015F00030E0C9010196877099274091B4014817DE
:10160000190671F40E942C071092B5011092B401D2
:1016100086E0E6EEF1E0DF011D928A95E9F7D2CF90
:1016200096E0929FD001939FB00D1124AA54BE4F13
:10163000FE01319601900D929A95E1F78093B501E4
:101640000E94B908BFCF819FC00111248A549E4FC8
:101650000E943E098823E9F0E091B4011E9FF00149
:101660001124EA54FE4F408151816281738184814B
:1016700095810E9469078091B40190E0019687707E
:1016800099278093B4018091B4019091B501891399
:10169000DACF2C96E3E00C94F02369857A858B856C
:1016A0009C850E9469078ECF682F809100019091E0
:1016B00001010E94DE1A0895682F80910001909127
:1016C00001010E94EC1A089580910001909101019E
:1016D0000E94FA1A089580910C028595859585954A
:1016E000089580910C028770089590910C02977074
:1016F00081E009F480E0089580912F02089590918F
:101700002F02892B80932F020895809590912F02AC
:10171000982390932F02089510922F02089590918C
:101720002E02892B80932E020895809590912E028F
:10173000982390932E02089510922E02089580917E
:101740000D02089508950E94A20B089590918502BC
:1017500092FF08C090910D02981721F080930D021E
:101760000E94A30B089580910D02882329F0109206
:101770000D0280E00E94A30B0895CF93DF93E091C8
:101780000001F091010180912F028083E09100011E
:10179000F0910101808190912E02892B808390919C
:1017A0000D02992381F0E0910001F0910101808107
:1017B000892B808380910001909101010E944A1A37
:1017C00081110E94B30BC0910001D091010140E250
:1017D00050E06CEE71E0CE010E941024892B59F08C
:1017E00080E2FE01ACEEB1E001900D928A95E1F746
:1017F000CE010E94F619DF91CF91089508950E94BD
:10180000FE0B08959091850292FF11C098E0899F88
:1018100090011124622B60930C020E94AE0780910C
:101820000C028595859585950E94FF0B08950E9471
:10183000AE07089510920C0280E00E94FF0B0895FD
:1018400090910C028095892380930C02282F277099
:1018500091F4282F082E000C330B9217130659F021
:101860009091850292FF07C08595859585950E9488
:10187000BA070E941A0C08959091850292FB2227C4
:1018800020F9281769F080FB92F9909385028091E6
:101890008402909185020E948E0C82E00E94200CAE
:1018A00008958091850282FB882780F991E089273D
:1018B0000E943C0C089581E00E943C0C089580E059
:1018C0000E943C0C08956FEF7FEF90E080E00E9453
:1018D0005224089590E080E00E942E24883E9E4F7E
:1018E00019F40E94EC13089580E0089582E090E0DE
:1018F0000E942624089583E090E00E942624089503
:10190000CF9384E090E00E942624C82F82E290E0EA
:101910000E942624982F8C2FCF910895CF93C92F02
:10192000682F84E090E00E9434246C2F82E290E0E3
:101930000E943424CF910895AB01BC018FE090E068
:101940000E9446240895AB01BC0183E190E00E940F
:101950004624089560E070E0CB010E94A30C089536
:1019600060E070E0CB010E949C0C0E94AA0C0895DC
:1019700068EE7EEF90E080E00E94522460E082E01A
:1019800090E00E94342460E083E090E00E943424E0
:101990001092B30160E084E090E00E94342464E09F
:1019A00082E290E00E94342460E085E090E00E94B2
:1019B000342460E086E090E00E9434246FEF87E0FA
:1019C00090E00E94342440E050E0BA0188E090E0CA
:1019D0000E94462460E08DE090E00E94342440E0C4
:1019E00050E0BA0188E190E00E94462460E087E17F
:1019F00090E00E94342440E050E0BA018CE190E095
:101A00000E94462470E060E080E290E00E94522450
:101A100040E050E0BA0188E190E00E94462480E076
:101A20000E9405140E9434140E94B00C08950E9474
:101A3000B80C0895682F8EE090E00E943424089539
:101A40000E94C81B60933E0270933F028093400245
:101A50009093410260933A0270933B0280933C0260
:101A600090933D020895089508950E94340D0895BD
:101A700008950E94380D089588EC9FE00E94DF19B8
:101A80000E94330D0E94350D089581E008950E9453
:101A9000450D0895089508950E944A0D0E944B0D2A
:101AA00008950E94E40F0E94660308950E94B31BEC
:101AB0000E9444140E94BC100E94510D0E94390DD6
:101AC0000895AAE0B0E0E7E6FDE00C94CA230E9486
:101AD000D21022E3822E22E0922E640110E0F60161
:101AE000E190F1906F01812F0E9407101F5F143069
:101AF00009F449C0E816F90691F38091420281FD8C
:101B00000E9410100E94470D782E10E0812F0E9435
:101B100007107C01F401A190B1904F018A159B053B
:101B200061F100E0CC24C394D12CAE24BF24C501C4
:101B30008C219D21892BC1F07720B1F00E831F836A
:101B400021E0C7018C219D21892B09F420E0288701
:101B50000E94BC1B8160782F9A8789874E815F81A4
:101B600068858A850E9492030F5FCC0CDD1C0C30C7
:101B7000F1F6F4013297F182E0821F5F143031F602
:101B80000E94200D22C0E816F90609F0B6CF0E9487
:101B9000BC1B8C018091300290913102081719070B
:101BA000A1F08FEF89838A831B820E94BC1B816016
:101BB000782F9D838C8349815A816B818D810E940E
:101BC000920310933102009330020E94F0120E949F
:101BD00079032A96EDE00C94E623CF93DF930E94DD
:101BE000E30EEC01811521E5920708F042C0811552
:101BF00030E5930708F09FC0883E910530F5803EA0
:101C0000910508F094C0883A910588F4853A9105C9
:101C100008F086C08130910509F489C0009709F465
:101C200086C0049708F083C0D0E0C0E080C08F3B3E
:101C30009105D0F7C85AD0E0CC0FDD1FC85BDE4F4E
:101C40000990D881C02DD46472C0811540E29407F8
:101C500050F4C11581E0D80708F069C0C03FD10534
:101C600018F3D06564C081159044F0F2DF70D06A3B
:101C70005EC0811535E5930718F5811544E5940795
:101C800008F085C0C11583E5D80708F06CC0C11500
:101C900022E5D20708F462C0CE018370992721E0C3
:101CA00030E002C0220F331F8A95E2F7C695C69531
:101CB00080E2C89FE0011124C22BD32BDC6837C01F
:101CC000811539E59307A8F4811548E5940708F0D4
:101CD00063C0C11586E5D80708F0A6CF8C2F0E94F7
:101CE000850FC82FD0E0DC2FCC27CC27DF71D06246
:101CF0001EC081152AE5920708F453C0905681153D
:101D0000904208F091CF8D2F8F710E94850F90E047
:101D1000982F882788279F719C012C2BE901E7CFFA
:101D2000C55AD0E0CA58DE4FC881D0E0D064CE0199
:101D3000DF91CF9108958370992721E030E002C0B0
:101D4000220F331F8A95E2F7C695C69540E2C49FDD
:101D5000E0011124C22BD32BDD68E9CFDC2FCC2787
:101D6000C16FD06AE4CFCE018370992721E030E0C3
:101D700002C0220F331F8A95E2F7C695C69540E24E
:101D8000C49FE0011124C22BD32BDA68D0CFD82F07
:101D9000CC27C46FD06ACBCFD82FCC27C06FD06AE6
:101DA000C6CF8F700E94850F34E0D695C7953A95BF
:101DB000E1F7CF709C2FEC01D069B9CF0E94471892
:101DC0000E94ED0D089582389105B9F1B0F4813388
:101DD000910509F47DC048F48932910509F46DC07C
:101DE0008A32910509F47BC008958533910509F481
:101DF0005FC08933910509F10895833E9105D9F1BA
:101E000038F4803E910529F1823E910579F10895DB
:101E1000863E9105D9F1873E910509F43EC0843E86
:101E2000910541F52091850221FF24C08091840213
:101E300084FD19C087EE90E00895209184022370FC
:101E400009F05AC02091850223FF14C089E290E076
:101E500008952091840220FD38C03091850230FF22
:101E600009C024FF43C090E080E0089520918402DF
:101E700022FDF7CF08952091840222FD3AC03091CF
:101E8000850230FD39C024FFF5CFEDCF20918402CB
:101E900023FFF0CF24FDE7CFCDCF2091840223FD97
:101EA0002EC03091850231FFEECF84EE90E0089590
:101EB0002091840225FFDECFC9CF2091840225FD29
:101EC00021C02091850223FFD5CF89E390E0D2CFB6
:101ED0002091840226FFCECF8AE290E008952091DF
:101EE000840226FFC7CF81E390E0089583EE90E05F
:101EF000089582EE90E0089580EE90E0089586EED9
:101F000090E0089585E390E008959091840292FF17
:101F100006C0282F28712830F9F4877F846093FF4A
:101F200006C0282F28712831F1F4877E8461209122
:101F3000850220FF06C0382F38713830D9F4877FEA
:101F4000816021FF06C0282F28712831D1F4877EB7
:101F5000816194FD877E0895282F24712430F9F63D
:101F60008B7F8860DCCF282F2471243101F78B7E92
:101F70008861DDCF382F3171313019F78E7F88605D
:101F8000E0CF282F2171213121F78E7E8861E1CFAA
:101F900080E008950E94630C08950E94D2108FE3A0
:101FA0009CE90197F1F700C000000E94D21080E088
:101FB0000E94071080FF04C00E94CA0F0E94071CE5
:101FC00008950E94CD0F08950E946A0C811102C0ED
:101FD0000E94170D0E94760C809342020E94800C92
:101FE00090938502809384020E94E10F0E947B0CF3
:101FF0000E947F078091B2010E949707089508957B
:102000000E94FF0F089508950E9403100895E82F7D
:10201000F0E0EE0FFF1FE257FD4F808191810895A0
:10202000089580EA8A95F1F7089500C008950E9406
:1020300011100895F894E82FE295EF70F0E031A1C7
:10204000282F2F7081E090E001C0880F2A95EAF7D1
:10205000982F9095932391A392A1892B82A3789492
:102060000895CF93DF9386EF0E941A1083E30E94B6
:102070001A1082E30E941A1086E30E941A10C9E720
:10208000D1E089918F3F11F00E941A1081E0C5388C
:10209000D807B9F7DF91CF910895AF92BF92DF9241
:1020A000EF92FF920F931F93CF93DF938C01D62E65
:1020B000C62FD0E0CE018B579E4F7C01FC012081C2
:1020C0002F3F09F44CC0F894E22FE295EF70F0E056
:1020D00031A12F7081E090E001C0880F2A95EAF7C6
:1020E000932F982B91A392A18095892382A3789412
:1020F0000E941510E9E7F1E041E050E0B12CA12C7D
:1021000021912F3FB1F1A22FA295AF70B0E0909630
:102110008C9190E02F7002C0959587952A95E2F7F3
:1021200080FD27C0CA01A82AB92A440F551F81E0A3
:10213000E538F80729F7F70180818F3F11F00E94F9
:102140001A1061E0A114B10409F460E08D2D0E9421
:102150001710CC0FDD1FC00FD11FB982A882DF91ED
:10216000CF911F910F91FF90EF90DF90BF90AF90B4
:10217000089590E080E0D7CF0E94311088E0EEE82B
:10218000F2E0DF01982F1D929A95E9F7E6E8F2E078
:10219000DF011D928A95E9F784E00E940D110E94EB
:1021A000DA020895A8E0B0E0E8EDF0E10C94D22363
:1021B0008E010F5F1F4F88E0F80111928A95E9F7B1
:1021C000F12C6F2DC8010E944D10F394F4E0FF1222
:1021D000F8CF48E050E0B80186E892E00E94102471
:1021E00021E0009709F420E0892B41F088E0F80114
:1021F000A6E8B2E001900D928A95E1F744E06EE81E
:1022000072E086E892E00E940E11182F0E94DD0213
:10221000812F2896E5E00C94EE230895CF92DF926B
:10222000EF92FF921F93CF93DF936C017B01C42F3A
:10223000222349F081E0809345020E94BC1B9093C9
:102240004402809343021091450211110AC010E02C
:10225000812FDF91CF911F91FF90EF90DF90CF9072
:10226000089580914302909144020E94D41B0597E7
:1022700070F3D0E0CC0FDD1FAE01B601C7010E94A4
:102280001024892B41F0AE01B601C7010E941D2424
:1022900010924502DDCF10E0FBCF0E94031E0E948A
:1022A000560D0E94101E08950E94151E0E94610D79
:1022B0000E942F1E08950E94551B0E94E91D0E9436
:1022C0003C0D0E944D110E9454110E944C0DFBCFF9
:1022D00080914C0280FF0DC06091070170E0660F95
:1022E000771F6038710570F56115710569F1862FEA
:1022F000089581FF07C06091070184E0689FB001E5
:102300001124EFCF6091070182FD0AC080914B023A
:102310008823A9F02091060160910701821710F02F
:1023200088E0ECCF869FC001112433E0880F991F0D
:102330003A95E1F7622F70E00E94A423D2CF68E0C3
:1023400070E0D5CF8FE7089581E0089580914C0229
:1023500080FF0CC06091030170E0759567957595DD
:1023600067956115710549F1862F089581FF06C0B3
:102370006091030170E075956795F3CF609103015B
:1023800082FD0BC090914A029923A1F06091020155
:1023900080910301961738F0682F70E0603871055E
:1023A00000F38FE70895899FC001112470E00E9417
:1023B000A423F4CF61E070E0D7CF81E00895803F9F
:1023C00031F40E9468118195809350020895813FF5
:1023D00019F40E946811F8CF823F31F40E9468110D
:1023E000819580934F020895833F19F40E946811EC
:1023F000F8CF893F29F40E94A611809351020895D5
:102400008A3F21F40E94A6118195F7CF8B3F31F4CA
:102410000E94A61181958093520208958C3F19F471
:102420000E94A611F8CF9CE0980F953070F4845F5D
:10243000990B21E030E001C0220F8A95EAF78091E4
:102440004E02822B80934E0208958D3F31F480918D
:102450004C02816080934C0208958E3F21F480915C
:102460004C028260F7CF8F3FB9F780914C028460B5
:10247000F1CF40914F02803F59F48091500287FF85
:102480000DC01092500241110BC010924B0208C0B7
:10249000813F81F48091500218169CF3442381F00F
:1024A0008091510290915202892B09F05AC01092EA
:1024B0004A020895823F49F447FFF0CF10924F023D
:1024C000809150028111ECCFE0CF833F19F41416B4
:1024D000ACF3E4CF90915102893F29F41916F4F638
:1024E00010925102DBCF8A3F19F497FFD7CFF8CF74
:1024F000909152028B3F29F497FFD0CF1092520255
:10250000CDCF8C3F19F41916CCF3C8CF9CE0980FAF
:10251000953090F4845F990B21E030E0B90102C05E
:10252000660F771F8A95E2F7CB01809590914E0256
:10253000892380934E02B2CF8D3F31F480914C02BB
:102540008E7F80934C02AACF8E3F21F480914C0263
:102550008D7FF7CF8F3F09F0A1CF80914C028B7F09
:10256000F0CF08950E94BC1B9C0190914F02809176
:102570005002982B21F03093490220934802909109
:10258000510280915202982B21F030934702209300
:1025900046028DE492E00E94101A089586E0EDE470
:1025A000F2E0DF011D928A95E9F710924B0210923A
:1025B0004A0210924C020895FC01828181110EC0E2
:1025C000838181110BC08481811108C091E08581D4
:1025D000811101C090E0892F8170089581E0FCCFC6
:1025E000A6E0B0E0E6EFF2E10C94D42386E0EDE45F
:1025F000F2E0DE01119601900D928A95E1F71092BA
:102600004F021092500210925102109252028B818E
:102610009C81892B89F080914802909149020E9407
:10262000D41BAC0190914B029923C9F18091080110
:102630008417150608F440C08D819E81892B91F086
:1026400080914602909147020E94D41BAC01909168
:102650004A02992309F471C0809104018417150678
:1026600008F479C0BE016F5F7F4F8DE492E00E9455
:102670000C1B811105C08DE492E00E94DC128111D7
:102680000E94B21286E0FE013196ADE4B2E0019004
:102690000D928A95E1F72696E3E00C94F0232091C1
:1026A00009018AE0289F900111242417350720F69C
:1026B0009F5F90934B0202C09F3FD1F71B81112374
:1026C00059F00E9468119FEF11160CF491E0899F58
:1026D000802D112480934F021C81112359F00E94F8
:1026E00068119FEF11160CF491E0899F802D112441
:1026F0008093500230914F02332309F49DCF2091F3
:102700005002222309F498CF45EB3403C001112471
:10271000992359F090934F0245EB24039001112423
:10272000332339F03093500287CF81E080934F02FA
:10273000F3CF81E0809350027FCF209105018AE0A2
:10274000289F900111242417350708F08BCF9F5F35
:1027500090934A0202C09F3FD1F71D81112359F087
:102760000E94A6119FEF11160CF491E0899F802D15
:102770001124809351021E81112359F00E94A61149
:102780009FEF11160CF491E0899F802D1124809306
:10279000520230915102332309F464CF2091520246
:1027A000222309F45FCF45EB3403C00111249923A0
:1027B00059F09093510245EB2403900111243323E7
:1027C00039F0309352024ECF81E080935102F3CF23
:1027D00081E08093520246CF83E290E00E9426245B
:1027E000823289F484E290E00E942624893059F4F0
:1027F00085E290E00E94262491E0843009F090E088
:10280000892F8170089580E0FCCFCF93C82F6FEFA0
:10281000811162E283E290E00E9434246FEFC111E3
:1028200069E084E290E00E9434246FEFC11164E01B
:1028300085E290E00E943424CF910895089586E2C5
:1028400090E00E942624682F70E090E080E00895D8
:102850000895CF93C62F0E9428146C2F86E290E033
:102860000E943424CF91089580E00E94051460E016
:1028700070E0CB010E9429140E94C1170E94A41885
:1028800081E00E94051408950E941E140E941F14E6
:102890000E9428140E94EC13811102C00E9434147B
:1028A0000895CF93FB01C281CC2309F19C012251F1
:1028B0003F452031310520F582510E94B418C0E017
:1028C0008C2FCF91089581E00E94AE0743E062E033
:1028D00081E00E94D002F3CF81E00E94BA0743E07A
:1028E00062E081E00E94D002EBCF82E0F6CF80313F
:1028F000FFE59F0789F381319F45B9F3C1E0E0CF40
:102900008031EFE59E07F9F281319F45C9F682E0FB
:10291000DBCF2FEFFC0120830895EF92FF920F93FE
:102920001F93CF93DF93EC01062FE881E150E33151
:1029300008F05DC0F0E0EA58FB4D0C94B823198212
:102940008AE08A83602FCE010E94BC1CCDB7DEB71F
:10295000E6E00C94ED238981823069F0833071F0D8
:102960008130D9F40E94C81B0E94BE236A837B83F6
:102970008C839D83E7CF0E941F14F6CF7E0110E069
:10298000812F0E940710F701928383831F5FF2E07B
:10299000EF0EF11C1430A1F7D5CF602FCE010E94AD
:1029A0008914D0CF89818230C1F76A817B818C8183
:1029B0009D810E94BE230E942914C4CF4B816A814D
:1029C00089810E9483179827892798279D838C8364
:1029D000B9CF2C813D813227232732274B816A8151
:1029E00089810E94A517AECF0E94C117ABCF8FEF90
:1029F0008883A8CF0E9455188983A4CF0E945718B6
:102A00009827892798279A8389839CCF6B8170E0C8
:102A100089819A81AE014C5F5F4F9827892798275B
:102A20000E945A188FCF6B8170E089819A81AE0124
:102A30004C5F5F4F9827892798270E947F1882CF85
:102A40000E94A4187FCF0E947117D6CF6B8170E0CF
:102A500089819A81AE014C5F5F4F9827892798271B
:102A60000E94FF176FCF6B8170E089819A81AE0160
:102A70004C5F5F4F9827892798270E94231862CFC1
:102A8000CF93DF93EC01FB018281882309F464C1B9
:102A9000C330FDE5DF07E0F5CA3F9CE5D90730F418
:102AA0009E0122503C4524313105D8F50E94800C0E
:102AB0009093850280938402C231ECE5DE0709F42D
:102AC0001FC108F06EC0C9308CE5D80709F4F2C008
:102AD00008F03FC0C530ECE5DE0709F4DBC058F56F
:102AE000C3308CE5D80709F4CDC008F0CFC0809181
:102AF00084028160C230DC4509F4AEC0809184025A
:102B0000909185020E948E0C0E942C0780E009C0E3
:102B1000C53AEDE5DE0751F238F4C1369DE5D90737
:102B200029F2DF91CF9108959E012D5A3D45233022
:102B30003105B8F7BBCF809184028062C730FCE5D5
:102B4000DF0709F489C008F4B1C080918402806471
:102B500083C0CD309CE5D90709F4BAC070F48091E8
:102B600084028E7FCB30FCE5DF0709F475C008F4E2
:102B7000A7C0809184028D7F6FC0CF309CE5D907BC
:102B800009F4B6C008F4A8C0C031FCE5DF0709F4B9
:102B9000B3C0C131DC4509F0B1CF809184028F7B95
:102BA0005BC0CF3F9CE5D90709F4B4C098F5CA3F94
:102BB000FCE5DF0709F472C0B8F4C4319CE5D9071D
:102BC00009F4B6C008F4A2C0C531DC4509F096CFBF
:102BD0008091840282FB992790F921E0922790FB53
:102BE00082F990FB83F938C0CC3F8CE5D80709F413
:102BF00077C008F457C0CD3FECE5DE0709F474C098
:102C0000809185028360CE3FDC4509F077CF8093C9
:102C1000850274CFC1368DE5D80709F496C068F4F3
:102C2000C130EDE5DE0709F48CC008F477C0C2308E
:102C3000DD4509F063CF80E085C0CD3A9DE5D90739
:102C4000E9F068F490918402892F8E7F90FF816073
:102C5000C53ADD4509F052CF809384024FCFCE3A7A
:102C60008DE5D80789F1CF3ADD4509F047CF90913E
:102C70008502892F877F93FF8860C9CF8091850265
:102C80008860C5CF809184028260E6CF8091840203
:102C90008460E2CF809184028860DECF80918502DB
:102CA0008160B5CF809185028260B1CF809184022E
:102CB0008061D2CF0E942C07809184028068CCCFA3
:102CC000809184028C60C8CF80918502877F9FCFDE
:102CD000809184028B7FC0CF80918402877FBCCF9C
:102CE000809185028E7F93CF809185028D7F8FCFDB
:102CF000809184028F7EB0CF809184028F7DACCF93
:102D00000E942C07809184028F77A6CF8091840245
:102D1000837FA2CF809185028C7F79CF80918502BD
:102D2000982F909591708E7F892B90FB81F96FCFB2
:102D30000E942C0790918402892F97FB87F9805875
:102D40008BCF81E00E941A0DD9CE90918402892FF9
:102D50008F7E94FF806180CF81E0E3CEB0E0A0E081
:102D6000E4EBF6E10C94D023E82FF0E0E45DFD4FB6
:102D7000D490282F26952695269530E0F901E45326
:102D8000FD4F0491877010E0082E02C0159507953D
:102D90000A94E2F701701127F901E454FD4FE49021
:102DA000F12C082E02C0F594E7940A94E2F791E022
:102DB000E922FF24F901E455FD4FC491D0E002C09F
:102DC000D595C7958A95E2F7C170DD2701151105E4
:102DD00019F081EE0E94CD03E114F10419F086EEA2
:102DE0000E94CD038D2D0E94CF04E114F10419F04F
:102DF00086EE0E945E040115110519F081EE0E9415
:102E00005E04CD2B19F08CE20E94CF04CDB7DEB763
:102E1000E7E00C94EC23EF92FF920F931F93CF9374
:102E2000DF93EC01162F0AE08881882309F454C04F
:102E3000813009F04EC08981813099F47E0122E011
:102E4000E20EF11C8A810E94CF04E7012196812FB6
:102E5000815050F3EFE9FFE03197F1F700C0000037
:102E6000F7CF823041F47E0182E0E80EF11C8A81C6
:102E70000E94CD03EACF833041F47E01E2E0EE0E02
:102E8000F11C8A810E945E04E0CF843011F021960B
:102E9000DDCF2A81229690E080E0AE014F5F5F4F48
:102EA0002053330B2A30310548F0019778F2EFE9CF
:102EB000FFE03197F1F700C00000F7CF089FB001A5
:102EC000099F700D1124C901860F971F2981EA01FE
:102ED000E4CF0E94AE16BACFCDB7DEB7E6E00C94D1
:102EE000ED2384E0089550E0440F551F98E1699F59
:102EF000400D511D112490E6899F400D511D112454
:102F0000CA01879608950F931F93CF93DF93843060
:102F1000C8F46430B8F44C30A8F40E9473178C01E4
:102F20000E942624C82FD0E0DC2FCC27C8010196B0
:102F30000E9426249E01282BC901DF91CF911F9169
:102F40000F91089590E080E0F8CF0F931F93CF93F7
:102F5000DF93122F032F843078F4643068F44C3000
:102F600058F40E947317EC01602F0E943424612FE3
:102F7000CE0101960E943424DF91CF911F910F91D1
:102F80000895B0E0A0E0E7ECF7E10C94CE239CEAD2
:102F9000C92E90E0D92ED0E0C0E07601B12C20C03F
:102FA0000E94620221E030E08C171D0641F03CF0E7
:102FB000F801EE0FFF1FEE0DFF1D25913491402FFC
:102FC0006B2D8C2F0E94A5170F5F1F4F0C30110522
:102FD00039F788E1E80EF11CB39484E0B81619F0D3
:102FE00010E000E0DDCF219680E6C80ED11CC43091
:102FF000D10599F6CDB7DEB7E9E00C94EA23EF925C
:10300000FF920F931F93CF93DF93EC018A017C0112
:10301000E60EF71ECE018796CE15DF0529F4CDB753
:10302000DEB7E6E00C94ED23C03821E0D20740F48F
:103030000E942624F80180830F5F1F4F2196EACF5C
:10304000F8011082F9CFB0E0A0E0E9E2F8E10C94D9
:10305000CF237C016A018C01060F171FEC01CE0102
:103060008796C017D10729F4CDB7DEB7E8E00C94F6
:10307000EB23C03821E0D20740F4FE01EE19FF092E
:10308000EC0DFD1D60810E9434242196E8CF462F6F
:10309000843040F4743030F46C3020F4672F0E9498
:1030A0008317089590E080E0089580E1089589E510
:1030B00092E00895EF92FF920F931F93CF93DF93C7
:1030C000EC018A017C01E60EF71ECE0189559E4F68
:1030D000CE15DF0529F4CDB7DEB7E6E00C94ED237D
:1030E000C93522E0D20740F40E942624F8018083EB
:1030F0000F5F1F4F2196E9CFF8011082F9CFB0E0A2
:10310000A0E0E5E8F8E10C94CF237C016A018C0192
:10311000060F171FEC01CE0189559E4FC017D1072E
:1031200029F4CDB7DEB7E8E00C94EB23C93522E0F3
:10313000D20740F4FE01EE19FF09EC0DFD1D608180
:103140000E9434242196E7CFCF93DF93C7EAD1E0E2
:1031500060E0CE010E9434242196C11584E0D80796
:10316000B9F7DF91CF910895A4E0B0E0EAEBF8E180
:103170000C94D023F82E8FE08F1548F18FEF93E059
:103180000E942624811123C007EA11E0F11023C018
:1031900019821A821B821C82DD24D39478018FEF5E
:1031A000E81AF80AC8010E94262489831A82882313
:1031B00071F09FEF980F9330D8F48A83D9820E5F15
:1031C0001F4FC7010E9426248B83811112C02496B1
:1031D000E7E00C94EC23011584E01807C1F3C80163
:1031E0000E942624811101C0FA940F5F1F4FCECF99
:1031F000870160E0CE0101960E940B17CFCFCF93DD
:10320000DF93EB0186319C4511F50E947C0B9A817E
:10321000992399F08A7A91E009F490E0909353020F
:10322000811109C089E20E94540B0E94BD0B80E00D
:10323000DF91CF91089585E3F6CF809153028111FC
:1032400004C089E20E945C0BF0CF85E3FBCF81E0F4
:10325000EFCF0F931F93CF93DF93C42FD22FFC0197
:1032600082818823C9F0409356020E94BC1B909330
:1032700055028093540280E28C0F883040F4C7706E
:1032800081E001C0880FCA95EAF70E94D804DF9157
:10329000CF911F910F91089510915602141332C0CF
:1032A00080915402909155020E94D41B883C910554
:1032B00048F5C0E2CD0F1D17B9F080E2810F8830CC
:1032C00040F4177081E001C0880F1A95EAF70E9458
:1032D000DF04C83048F481E09D2F977001C0880F4B
:1032E0009A95EAF70E94D804802F0E94CF04C83034
:1032F00070F6D77081E001C0880FDA95EAF70E9476
:10330000DF04C5CF80E28C0F883008F6C77081E0FB
:1033100001C0880FCA95EAF7F2CF0F939C01CB0149
:10332000233F4CE5340759F1A8F4283DFCE53F075D
:1033300001F1293D4CE53407D1F1273D3C4591F49D
:1033400006E221EE41EE67ED7CE50E94291980E05E
:103350000F910895253FFCE53F07E9F0B0F0263FC7
:103360003C45F9F0FC018281882339F11092560224
:10337000EFCF07E225EE45EE68ED7CE5E6CF06E20D
:1033800021EE40EE63EF7CE5E0CF07E225EE44EE70
:1033900064EF7CE5DACF06E221EE42EE65EF7CE5F4
:1033A000D4CF07E225EE46EE66EF7CE5CECF08E20D
:1033B00021E045EE69ED7CE5C8CF81E0C9CF90936F
:1033C000990180939801089590935C0280935B0229
:1033D0000895E0915B02F0915C02309729F0019032
:1033E000F081E02D0995089580E00895E0915B0259
:1033F000F0915C02309799F020911601222359F048
:103400002091840227FF07C0DC012C9111962C9398
:10341000119726E02C930280F381E02D0995089501
:10342000E0915B02F0915C02309739F022E0DC0120
:103430002C930480F581E02D09950895209159027F
:1034400030915A022817390771F090935A028093ED
:103450005902E0915B02F0915C02309721F0068006
:10346000F781E02D09950895209157023091580277
:103470002817390771F09093580280935702E09112
:103480005B02F0915C02309721F00084F185E02D21
:1034900009950895FC01329680911601882321F048
:1034A000809184029EE187FF96E080E0915008F4CD
:1034B000089521912223D1F38F5FF8CF662301F184
:1034C000209116012223F1F02091840227FF1AC0D7
:1034D000462F4695469546954E3190F4677021E00B
:1034E00030E002C0220F331F6A95E2F7840F911D6E
:1034F000FC01828190E02823392381E0232B69F4A9
:1035000080E00895FC01329608962191261721F05B
:10351000E817F907D1F7F4CF81E008959C01FC0189
:1035200032969FEF80E04191461751F09F3F19F48A
:10353000411101C0982F8F5F8630A9F79F3F09F492
:103540000895290F311D97FD3A95F9016283089579
:10355000FC01329608962191261303C0DF011197D2
:103560001C92E817F907B9F70895E62FE695E69556
:10357000E695EE3168F4E80FF92FF11D677021E050
:1035800030E001C0220F6A95EAF78281822B8283A4
:103590000895E62FE695E695E695EE3170F4E80F8E
:1035A000F92FF11D677021E030E001C0220F6A950C
:1035B000EAF720958281282322830895209116011D
:1035C000222339F02091840227FF03C00E94B51AFC
:1035D00008950E948E1A089520911601222339F031
:1035E0002091840227FF03C00E94C91A08950E94F7
:1035F000A81A0895FC01329680911601882351F093
:103600008091840287FF06C08EE1DF011D928A95BA
:10361000E9F7089586E0F9CF46E050E00E941024D3
:1036200021E0892B09F420E0822F089508950E945B
:10363000161B0895811106C081E080935D020E94EF
:10364000171B089582E0F9CF83E080935D020E940A
:10365000171B08950E941A1B089581E080935D0254
:103660000E94171B08950E942D1B08950895089528
:103670000E94371B0895089508950E94361B0895EF
:10368000CF930E943B1B0E94D2100E943C1BC0E0C3
:103690008C2F0E940710892B31F4CF5FC430C1F703
:1036A00080E0CF91089581E0FCCF85B7806885BF29
:1036B00085B7806885BF08951F921FB61F92112499
:1036C0008F939F93AF93BF9380915E02811113C03C
:1036D0008091960290919702A0919802B0919902E0
:1036E0004196A11DB11D8093960290939702A093DD
:1036F0009802B0939902BF91AF919F918F911F90C3
:103700001FBE1F90189580919E02843031F10E9457
:10371000530310925E0288E190E020E40FB6F89423
:10372000A895809360000FBE2093600083B7817FCF
:10373000846083BF83B7816083BF7894889583B7A3
:103740008E7F83BF0FB6F894A89580916000886142
:1037500080936000109260000FBE08950E942C07B5
:103760000E945803089582E084BD93E095BD9AEFCE
:1037700097BD80936E0008952FB7F89480919602BC
:1037800090919702A0919802B09199022FBF08954D
:103790002FB7F894609196027091970280919802E9
:1037A000909199022FBF08959C014FB7F894809192
:1037B000960290919702A0919802B09199024FBF02
:1037C000821B930B089578941F921FB61F921124A9
:1037D0008F939F93AF93BF9380919602909197029E
:1037E000A0919802B09199020196A11DB11D8093FC
:1037F000960290939702A0939802B0939902BF917A
:10380000AF919F918F911F901FBE1F90189587E7D2
:1038100097E7909301088093000888E19AE00FB63B
:10382000F894A895809360000FBE90936000FFCF3E
:1038300088E19AE00FB6F894A895809360000FBED7
:1038400090936000FFCF80918202089508959C01BB
:1038500084E08093E9009FEF8091E800915085FD1E
:1038600006C085ED8A95F1F700009111F5CF8091A2
:10387000E80085FF0CC050E040E066E070E0C90160
:103880000E94CE1E8091E8008E778093E800089514
:10389000CF93DF93EC01809116018823B1F18091E1
:1038A000840287FF32C060E284E08093E9008FEFFA
:1038B0009091E800815095FD06C095ED9A95F1F73D
:1038C00000008111F5CF8091E80085FF1BC0809139
:1038D000160170E050E040E0811104C050E040E08B
:1038E00068E070E0CE010E94CE1E8091E8008E77E5
:1038F0008093E80080E2FE01A2E6B2E001900D9222
:103900008A95E1F7DF91CF91089568E081E0CDCF0E
:1039100080935F02709361026093600280919E02C7
:103920008430F9F48093E9008FEF9091E8008150A2
:1039300095FD06C095ED9A95F1F700008111F5CF40
:103940008091E80085FF0DC050E040E063E070E04A
:103950008FE592E00E94CE1E8091E8008E778093E2
:10396000E8000895BC0184E00E94881C0895BC0111
:1039700083E00E94881C0895CF93FC01603221F5FA
:1039800080919E02843001F5C091E900CF702091B2
:10399000EC00922F917020FD90E8C92B82E080937B
:1039A000E9008091E80080FF0CC050E040E060E258
:1039B00070E0CF010E94CE1E8091E8008E77809348
:1039C000E800CF70C093E900CF91089580919D02E7
:1039D000811109C00E94AD200E940A218091E2005D
:1039E00084608093E200089510929D0208950E94E1
:1039F0002D1B089560919A0281E0611101C080E061
:103A00000E94241B089590919E0281E0943009F059
:103A100080E060919A020E942A1B089542E061ECC6
:103A200081E00E94292042E261EC84E00E9429208A
:103A300042E261EC82E00E94292042E260EC83E0F5
:103A40000E94292090919E0281E0943009F080E04C
:103A500060919A020E941A1B08958091A0028330FF
:103A600009F463C030F48130E1F1823009F4A0C080
:103A700008958A3009F48CC08B3009F471C0893004
:103A800009F052C080919F02813209F04DC08091AF
:103A9000A3029091A402009719F0029709F044C084
:103AA0008091E800877F8093E8008091E80082FFA2
:103AB00037C09091F3008091F200029731F4809129
:103AC000F100813011F0863021F48091F100809373
:103AD00082028091E8008B778093E8000E945D204D
:103AE00023C080919F02813AF9F48091E800877F9A
:103AF0008093E8008091A3029091A402892B61F445
:103B000060E282E692E070E00E946C1F8091E80023
:103B10008B778093E800089560E090E080E0F3CF39
:103B200080919E028111C1CF089580919F02813AB8
:103B3000D9F78091A3029091A402892BA9F78091D3
:103B4000E800877F8093E8008091E80080FFFCCF49
:103B5000809116018093F1008091E8008E77BCCFB0
:103B600080919F02813201F78091A3029091A4027B
:103B7000892BD1F68091E800877F8093E8000E942E
:103B80005D208091A102809316010E942C07089568
:103B900080919F02813241F68091E800877F809377
:103BA000E8000E945D208091A20280938302089524
:103BB00080919F02813A09F0B7CF8091E800877F1A
:103BC0008093E8008091E80080FFFCCF8091830221
:103BD000C1CF84B7877F84BF0FB6F894A895809132
:103BE0006000886180936000109260000FBE80E8E2
:103BF00090E00FB6F89480936100909361000FBE3F
:103C00000E94331B08950E94AD200E940A21E2EE1B
:103C1000F0E080818460808378940E9489230895F5
:103C20008AE091E00E94E419089580919E02853017
:103C300031F480919E02853019F00E94AE1B0895E8
:103C40000E94831B80919C02882399F30E94401B51
:103C5000882379F30E94B81E0E942C07EACFA0E2C5
:103C6000B0E0E5E3FEE10C94D52380919E02843020
:103C700009F583E08093E9008091E80082FF1AC093
:103C80008091E80090E085FF09C050E040E060E2EC
:103C900070E0CE0101960E941D1F91E08091E80026
:103CA0008B778093E800992329F060E2CE0101969A
:103CB0000E948D14A096E2E00C94F1230E94611EF4
:103CC0000895292F33272330310521F168F421305D
:103CD000310509F443C02230310509F444C090E0B5
:103CE00080E030E020E026C02132310551F122325F
:103CF0003105A9F76330710590F7FB01EE0FFF1F47
:103D0000E457FE4F2081318167577E4FFB01808150
:103D100090E010C099278130910581F0009729F03B
:103D20000297E9F6ECEDF2E002C0ECEFF2E08491EC
:103D300090E09F01FA01318320830895ECEEF2E0D8
:103D4000F6CF6330710558F6660F771FFB01EE560C
:103D5000FE4F2081318189E090E0ECCF82E190E05C
:103D60002BE533E0E7CF8BE590E020E033E0E2CFD6
:103D700080E189BD82E189BD09B400FEFDCF80915B
:103D8000D8008F7D8093D8008091E000826080937E
:103D9000E0008091E00081FDFCCF0895AF92BF92DA
:103DA000CF92DF92FF920F931F93CF93DF936C011B
:103DB000EB018A010E947C20F82E811123C001159D
:103DC000110539F0F80180819181C81BD90BC80E0B
:103DD000D91EB12CA12C2097A9F08091E80085FD77
:103DE00022C08091E8008E778093E80001151105CC
:103DF000A1F0F80180819181A80EB91EB182A08244
:103E000085E0F82E8F2DDF91CF911F910F91FF90BC
:103E1000DF90CF90BF90AF9008950E947C208823C0
:103E2000D1F2F82EEFCFF60181916F018093F1006E
:103E30002197FFEFAF1ABF0ACECFAF92BF92CF92BA
:103E4000DF92FF920F931F93CF93DF936C01EB01EF
:103E50008A010E947C20F82E811123C001151105D2
:103E600039F0F80180819181C81BD90BC80ED91E89
:103E7000B12CA12C2097A9F08091E80085FD22C0EB
:103E80008091E8008B778093E80001151105A1F07F
:103E9000F80180819181A80EB91EB182A08285E0CF
:103EA000F82E8F2DDF91CF911F910F91FF90DF9012
:103EB000CF90BF90AF9008950E947C208823D1F2CC
:103EC000F82EEFCF8091F100F60181936F012197D9
:103ED000FFEFAF1ABF0ACECFFC018091A5029091EF
:103EE000A60286179707A0F06115710529F4909135
:103EF000E8009E779093E80090E06115710551F419
:103F0000911108C08091E80082FF34C080E00895DC
:103F1000BC01F2CF80919E028823C1F18530C1F1AE
:103F20008091E80083FD30C08091E80082FDEACFF7
:103F30008091E80080FFE1CF8091F3002091F200B2
:103F4000382F6115710519F02830310558F091E0CE
:103F50002830310509F090E02091E8002E77209379
:103F6000E800CBCF81918093F100615071092F5F00
:103F70003F4FE7CF80919E02882341F0853041F08A
:103F80008091E80083FFBECF81E0089582E008952C
:103F900083E00895FC018091A5029091A602861706
:103FA0009707A0F06115710529F48091E8008E77DC
:103FB0008093E80090E06115710551F4911108C0FB
:103FC0008091E80082FF35C080E00895BC01F2CF07
:103FD00080919E028823C9F18530C9F18091E80063
:103FE00083FD31C08091E80082FDEACF8091E80036
:103FF00080FFE1CF8091F3002091F200382F61150E
:10400000710519F02830310558F091E0283031055C
:1040100009F090E08091E8008E778093E800CBCFA4
:1040200084918093F1003196615071092F5F3F4F69
:10403000E6CF80919E02882341F0853041F0809147
:10404000E80083FFBDCF81E0089582E0089583E01A
:104050000895982F973028F08F708093E90081E0C1
:1040600008959093E900242F762F50E0981731F0AF
:104070007091EC002091ED005091F00021FD02C004
:104080009F5FE8CF3091EB003E7F3093EB003091A3
:10409000ED003D7F3093ED003091EB0031603093C7
:1040A000EB007093EC002093ED005093F000209112
:1040B000EE0027FDE5CF80E0089580919F0287FF05
:1040C00013C08091E80082FF06C08091E8008B77E2
:1040D0008093E80004C080919E028111F2CF089580
:1040E00080919E028823D9F38091E80080FFF8CF69
:1040F0008091E8008E77ECCF2091E4003091E500CC
:1041000095E6A9012091EC00822F817020FF06C066
:104110008091E80080FF06C080E008952091E800CB
:1041200022FD1AC080919E02882389F0853089F093
:104130008091EB0085FD0FC02091E4003091E500F7
:1041400042175307F9F29150E1F684E0089582E0B6
:10415000089583E0089581E008950E941C210E9443
:104160002421E0EEF0E0808181608083E8EDF0E0E2
:1041700080818F77808319BCA7EDB0E08C918E7F12
:104180008C9380818F7E808310929D0208950F937F
:104190001F93CF93DF930E941C210E942421C8ED1E
:1041A000D0E088818F778883888180688883888140
:1041B0008F7D888319BC10929E0210929A021092F1
:1041C0009C0210929B0200EE10E0F80180818B7F30
:1041D000808388818160888342E060E080E00E9483
:1041E0002920E1EEF0E080818E7F8083E2EEF0E036
:1041F000808181608083808188608083F8018081F4
:104200008E7F8083888180618883DF91CF911F9129
:104210000F910895E8EDF0E080818F7E8083E7EDD7
:10422000F0E080818160808384E082BF81E08093C0
:104230009D020E94C7200895E8EDF0E080818E7F06
:1042400080831092E20008951092DA001092E1004B
:1042500008951F920F920FB60F9211242F933F9340
:104260004F935F936F937F938F939F93AF93BF937E
:10427000EF93FF938091E10082FF0BC08091E200F9
:1042800082FF07C08091E1008B7F8093E1000E9454
:1042900088238091DA0080FF19C08091D80080FFC8
:1042A00015C08091DA008E7F8093DA008091D9006A
:1042B00080FF96C080E189BD82E189BD09B400FE1E
:1042C000FDCF81E080939E020E94E61C8091E10078
:1042D00080FF19C08091E20080FF15C08091E2004C
:1042E0008E7F8093E2008091E20080618093E20003
:1042F0008091D80080628093D80019BC85E08093BB
:104300009E020E94FA1C8091E10084FF2BC08091E4
:10431000E20084FF27C080E189BD82E189BD89B5C3
:10432000982F917080FFFBCF8091D8008F7D809374
:10433000D8008091E1008F7E8093E1008091E200BF
:104340008F7E8093E2008091E20081608093E200A2
:1043500080919A02882309F449C084E080939E02E8
:104360000E94031D8091E10083FF29C08091E2003B
:1043700083FF25C08091E100877F8093E10082E088
:1043800080939E0210929A028091E1008E7F80932A
:10439000E1008091E2008E7F8093E2008091E20054
:1043A00080618093E20042E060E080E00E9429208A
:1043B0008091F00088608093F0000E94F71CFF91CC
:1043C000EF91BF91AF919F918F917F916F915F918D
:1043D0004F913F912F910F900FBE0F901F90189506
:1043E00019BC10929E020E94F41C70CF8091E300D1
:1043F00087FD93E090939E02B3CF1F920F920FB66A
:104400000F9211242F933F934F935F936F937F935A
:104410008F939F93AF93BF93CF93DF93EF93FF93CC
:10442000D091E900DF708091EC00C82FC17080FD51
:10443000C0E81092E9008091F000877F8093F0003F
:1044400078940E9441221092E9008091F0008860E7
:104450008093F000CD2BCF70C093E900FF91EF91D6
:10446000DF91CF91BF91AF919F918F917F916F918C
:104470005F914F913F912F910F900FBE0F901F9022
:104480001895AAE2B0E0E7E4F2E20C94D4238FE9B5
:1044900092E02091F100FC012193CF01F2E0873AF4
:1044A0009F07B9F70E942D1D8091E80083FF1EC170
:1044B00080919F029091A0029A3008F017C1E92FD5
:1044C000F0E0E757FB4D0C94B823803899F0823820
:1044D00009F00CC18091A3028F70873008F006C1EB
:1044E0008093E9008091EB0085FB882780F910928A
:1044F000E90006C080919B0290919C02911182601C
:104500009091E800977F9093E8008093F1001092DB
:10451000F1008091E8008E77E5C0882309F4D3C0CC
:10452000823009F0E3C08091A1028111D6C0809150
:10453000A3028F702FEF280F263008F0D7C080938A
:10454000E9002091EB0020FFC8C0933031F4809146
:10455000EB0080628093EB00C0C09091EB00906113
:104560009093EB0021E030E001C0220F8A95EAF73A
:104570002093EA001092EA008091EB008860EACF75
:104580008111B4C01091A1021F778091E30080785F
:10459000812B8093E3008091E800877F8093E8007F
:1045A0000E945D208091E80080FFFCCF8091E300B5
:1045B00080688093E30082E0111183E080939E0283
:1045C00095C08058823008F091C08091A1029091EE
:1045D000A2028C3D23E09207A1F583E08A838AE260
:1045E00089834FB7F894DE01139620E03EE051E254
:1045F000E32FF0E050935700E49120FF03C0E295D1
:10460000EF703F5FEF708E2F90E0EA30C0F0C796FA
:104610008D939D932F5F243159F74FBF8091E80010
:10462000877F8093E8006AE270E0CE0101960E94E5
:104630006C1F8091E8008B778093E80057C0C0968C
:10464000E7CF6091A3027091A402AE014F5F5F4F6C
:104650000E945E1EBC01892B09F448C09091E800BD
:10466000977F9093E80089819A810E94CA1FE1CFC9
:104670008038E1F58091E800877F8093E8008091A1
:104680009A028093F10045CF811130C09091A10230
:10469000923060F58091E800877F8093E8009093E6
:1046A0009A020E945D2080919A02882311F084E092
:1046B00005C08091E30087FDFACF81E080939E02E0
:1046C0000E940E1D13C08091A102813079F481E017
:1046D000933009F080E080939C021092E900809171
:1046E000E800877F8093E8000E945D208091E800C9
:1046F00083FF0AC08091E800877F8093E800809163
:10470000EB0080628093EB00AA96E3E00C94F02328
:104710000895CF9380919E028823A1F0C091E90073
:10472000CF709091EC00892F817090FD80E8C82BAC
:104730001092E9008091E80083FD0E944122CF7031
:10474000C093E900CF91089597FB072E16F40094CB
:1047500007D077FD09D00E94FC2307FC05D03EF46A
:10476000909581959F4F0895709561957F4F08951D
:10477000EE0FFF1F0590F491E02D0994692796270D
:10478000692778278727782708952F923F924F929D
:104790005F926F927F928F929F92AF92BF92CF92D1
:1047A000DF92EF92FF920F931F93CF93DF93CDB7DA
:1047B000DEB7CA1BDB0B0FB6F894DEBF0FBECDBF52
:1047C00009942A88398848885F846E847D848C8423
:1047D0009B84AA84B984C884DF80EE80FD800C812C
:1047E0001B81AA81B981CE0FD11D0FB6F894DEBF0F
:1047F0000FBECDBFED010895AA1BBB1B51E107C041
:10480000AA1FBB1FA617B70710F0A61BB70B881F60
:10481000991F5A95A9F780959095BC01CD010895EF
:10482000FB01DC0104C08D910190801921F44150FD
:104830005040C8F7881B990B0895FB01DC0102C0AA
:1048400001900D9241505040D8F70895F999FECF4C
:1048500092BD81BDF89A992780B50895A8E1B0E08E
:1048600042E050E00C945A24262FF999FECF92BDD5
:1048700081BDF89A019700B4021639F01FBA20BD25
:104880000FB6F894FA9AF99A0FBE08950396272F57
:104890000E9435240E943424252F0E943524242F81
:1048A0000C9435240196272F0E9435240C9434242F
:1048B000DC01CB01FC01F999FECF06C0F2BDE1BDE0
:1048C000F89A319600B40D9241505040B8F70895CF
:1048D000F894FFCF2105210552055205DF05FB05A0
:1048E0008105810506066D067C067C069F14AB14C7
:1048F000D214DE14E914F414F714F714F714F714AF
:10490000F714FA14FE140615131520152315261591
:10491000331565228D2276238D227623C022E12253
:0649200076233823442336
:104926000E02280850011E0A1401231C481C271CCD
:10493600B71CB21C261C01E200E900EA00B500B66D
:1049460000B700CD008301CC008A019201940121B9
:1049560002230224022502260227022A02B300B4F9
:10496600006F007000818283E200E900EA00B50072
:10497600B600B700CD008301CC008A0192019401F4
:104986002102230224022502260227022A02B3005C
:10499600B4006F007000818283F4F53534C69766E3
:1049A6009490919293F63332364022B645046D03C5
:0849B6008F0312032B034B03D6
:00000001FF
